:100000000C9474010C9491010C9491010C94910145
:100010000C9491010C9491010C9491010C94910118
:100020000C9491010C9491010C9491010C94910108
:100030000C9491010C9491010C9491010C949101F8
:100040000C9491010C9491010C9491010C949101E8
:100050000C9491010C94AF060C9491010C949101B5
:100060000C9491010C949101808183848687898A04
:100070008C8E8F9192949597989A9B9D9EA0A2A307
:10008000A5A6A7A9AAACADAFB0B2B3B5B6B7B9BA79
:10009000BCBDBEC0C1C2C4C5C6C8C9CACBCDCECF07
:1000A000D0D2D3D4D5D6D7D9DADBDCDDDEDFE0E1C0
:1000B000E2E3E4E5E6E7E8E9EAEAEBECEDEEEEEFB1
:1000C000F0F1F1F2F3F3F4F5F5F6F6F7F8F8F9F9E3
:1000D000FAFAFAFBFBFCFCFCFDFDFDFDFEFEFEFE5C
:1000E000FEFFFFFFFFFFFFFF0000891112239B327D
:1000F0002446AD573665BF74488CC19D5AAFD3BEF8
:100100006CCAE5DB7EE9F7F88110080193331A2207
:10011000A5562C47B7753E64C99C408DDBBF52AED7
:10012000EDDA64CBFFF976E802218B3010029913E7
:100130002667AF763444BD554AADC3BC588ED19FB7
:100140006EEBE7FA7CC8F5D983310A2091121803C7
:10015000A7772E66B5543C45CBBD42ACD99E508F97
:10016000EFFB66EAFDD874C904428D5316619F7097
:100170002004A9153227BB364CCEC5DF5EEDD7FC77
:100180006888E1997AABF3BA85520C4397711E6087
:10019000A1142805B3373A26CDDE44CFDFFD56EC57
:1001A000E9986089FBBB72AA06638F7214409D5167
:1001B0002225AB343006B9174EEFC7FE5CCCD5DD37
:1001C0006AA9E3B8788AF19B87730E6295501C4147
:1001D000A3352A24B1163807CFFF46EEDDDC54CD17
:1001E000EBB962A8F99A708B088481951AA793B627
:1001F0002CC2A5D33EE1B7F04008C919522BDB3A17
:10020000644EED5F766DFF7C899400859BB712A6E6
:10021000ADD224C3BFF136E0C1184809D33B5A2AF6
:10022000E55E6C4FF77D7E6C0AA583B418869197C6
:100230002EE3A7F23CC0B5D14229CB38500AD91BD6
:10024000666FEF7E744CFD5D8BB502A499961087A6
:10025000AFF326E2BDD034C1C3394A28D11A580BB6
:10026000E77F6E6EF55C7C4D0CC685D71EE597F476
:100270002880A1913AA3B3B2444ACD5B5669DF7896
:10028000600CE91D722FFB3E8DD604C79FF516E466
:10029000A9902081BBB332A2C55A4C4BD7795E6876
:1002A000E11C680DF33F7A2E0EE787F61CC495D546
:1002B0002AA1A3B03882B193466BCF7A5448DD5956
:1002C000622DEB3C700EF91F8FF706E69DD414C526
:1002D000ABB122A0B9923083C77B4E6AD5585C4936
:1002E000E33D6A2CF11E780F11241FBECFEFD8E03A
:1002F000DEBFCDBF11E0A0E0B1E0E8E3F6E102C06F
:1003000005900D92A231B107D9F718E0A2E1B1E052
:1003100001C01D92AC33B107E1F70E94D5090C94DE
:100320001A0B0C9400000C94610878948CE294E011
:100330000E940A0343E951E06CE274E088E095E032
:100340000E9448078AEF94E00E94C301E6E3F8E0C8
:100350008AEF94E09383828391838083AC016CE283
:1003600074E088E095E00C9454089091C00095FFEB
:10037000FCCF8093C60008958091C00087FFFCCF1A
:100380008091C6000895CF93DF93CDB7DEB72E9747
:100390000FB6F894DEBF0FBECDBFDC018EE0FD01CD
:1003A000982F11929A95E9F71092C50097E69093CD
:1003B000C400E0ECF0E090819D7F908396E0909304
:1003C000C20098E19093C1009E012F5F3F4FF90159
:1003D00011928A95E9F783E08C8385EB91E09A8707
:1003E00089878CEB91E09C878B879EE0F9010190D7
:1003F0000D929A95E1F72E960FB6F894DEBF0FBED8
:10040000CDBFDF91CF910895811106C08091C000CA
:10041000881F8827881F089580E008958091C00074
:1004200087FF03C08091C60008958FEF08950F9352
:100430001F93CF93DF93182FC0912C08D0912D08D4
:10044000FE01E959FF4F8081811124C080E490E0D2
:100450009E8F8D8F1C8E1B8E1A8E01E00083299A31
:100460002091090130910A0140910B0150910C013A
:10047000A0EBB4E00E94F4096056704F8F4F9F4F7D
:1004800020E43FE140E050E00E94FF093B8B2A8BD3
:10049000009313010FB7F8942091050130910601E4
:1004A0004091070150910801A0EBB4E00E94F409CB
:1004B0006056704F8F4F9F4F20E43FE140E050E087
:1004C0000E94FF093D8B2C8B0FBFE0912C08F0910F
:1004D0002D084FB7F89423A134A1878D90A1281738
:1004E000390739F425A136A181A192A1281739072E
:1004F00079F065A176A123A134A12150310991E0C1
:1005000080E06217730709F090E0292F382F02C0AE
:1005100021E030E04FBF232BC1F6E0912C08F09191
:100520002D082FB7F894A5A1B6A11C9345A156A1FB
:1005300081A192A14817590719F4878D90A103C092
:1005400085A196A1019696A385A32FBFDF91CF9198
:100550001F910F910895E0912C08F0912D084FB74D
:10056000F894EB58FF4F24813581868197814FBFE6
:1005700028173907E9F0E0912C08F0912D089FB772
:10058000F894EB58FF4FA481B58122813381A217E3
:10059000B30719F42081318105C0A481B5819D0183
:1005A0002F5F3F4F358324838C919FBF90E0089548
:1005B0008FEF9FEF089581E080931201089581E00D
:1005C000809312011092800089E18093810081E87C
:1005D00096E0909387008093860080911201882393
:1005E00021F080E480937C0002C010927C00389857
:1005F000409880917E00816080937E0087E08093A8
:100600007B008CEE80937A008AB1886F8AB9219A38
:10061000229A08950F931F93CF93DF93CDB7DEB740
:100620002E970FB6F894DEBF0FBECDBF8C018AECBB
:10063000D8011D928A95E9F710932D0800932C0894
:1006400080E490E0F801968F858FC80180599F4F14
:10065000E859FF4F918380839783868395838483B2
:100660000496938382830996D801AB58BF4F1196A5
:100670009C938E9317969C938E93169715969C93A6
:100680008E931497CF9613969C938E9312978559B9
:100690009109D80190969C938E935F9796969C9320
:1006A0008E93959794969C938E939397CF969296CC
:1006B0009C938E93919784E090E0A681B7811C92E1
:1006C00046815781228133814217530719F42081D3
:1006D000318104C0268137812F5F3F4F37832683C6
:1006E000019759F70E94DF028EE0FE013196DF018B
:1006F000982F1D929A95E9F793E09C8327E132E0C9
:100700003A8729872BEA32E03C872B87D801019072
:100710000D928A95E1F72E960FB6F894DEBF0FBEC4
:10072000CDBFDF91CF911F910F9108950F931F932C
:10073000CF93DF93E0912C08F0912D0825A136A1ED
:1007400034A323A3EC018C01060F171FC017D10798
:1007500021F089910E941702F9CFDF91CF911F916B
:100760000F910895DC0156968C9156978111ECC03B
:1007700058968C9158978111A2C093964D915C9197
:10078000949795962D913C9196974217530739F47B
:1007900054962D913C915597232B09F460C059969E
:1007A0009C915997911103C05A961C925A9791E0C7
:1007B00059969C93599752962D913C915397211598
:1007C000310599F593964D915C91949795962D915D
:1007D0003C9196974217530759F454962D913C91AA
:1007E00055972150310955963C932E93549723C029
:1007F0009396ED91FC91949791962D913C919297BF
:10080000E217F30729F45F962D913C91909707C06A
:100810009396ED91FC9194979F012F5F3F4F949693
:100820003C932E939397908107C0215031095396A2
:100830003C932E9352979EE757969C9357975796C3
:100840009C9157979B3189F593964D915C91949724
:1008500095962D913C9196974217530739F4109233
:100860001301A959BF4F1C92299808959396ED91B1
:10087000FC91949791968D919C919297E817F90726
:1008800029F45F968D919C91909706C09396ED9177
:10089000FC919497CF01019694969C938E93939795
:1008A000808157968C93579706C09E57923018F4C4
:1008B00059961C92599781E058968C93589759965F
:1008C0008C9159975D962D913C915E978823A9F064
:1008D0005A968C915A97853080F05A961C925A9766
:1008E0002034310519F080E490E002C085E790E003
:1008F0005E969C938E935D9723C058968C915897E3
:1009000057969C915797982341F05A969C915A97E5
:100910009F5F5A969C935A970FC05A961C925A976B
:100920002034310519F020E430E002C025E730E042
:100930005E963C932E935D97880F58968C935897AC
:1009400088E056968C9356975D96ED91FC915E9754
:100950005B968D919C915C97E80FF91F9F01317018
:100960005C963C932E935B9756968C91569781504C
:1009700056968C93FF27E038F10530F08FEF90E02A
:10098000AC014E1B5F0BFA01E859FF4F84912F3FDA
:10099000310511F008F080950895EF92FF920F93C2
:1009A0001F93CF93DF93FC018C0101541F4FD8019B
:1009B0004D915C911197129711965C934E93A555AA
:1009C000B10914968D919C91159712962D913C9199
:1009D00013978217930721F42D913C91119707C02B
:1009E00014968D919C9115979C012F5F3F4F159602
:1009F0003C932E931497EC01288126029001112438
:100A0000C9019595879595958795E8019983888380
:100A10007F01D3ECED0EF11CE701288139818F01B4
:100A20000F531F4FE80139832883840F951F359595
:100A30002795820F931FE70199838883AF014B535A
:100A40005F4F21E0181619060CF420E0EA018881B6
:100A5000880F822B888316968D919C911797EC01B5
:100A6000688316962D913C91179712968D919C91C3
:100A700013972817390721F48D919C91119705C080
:100A800016968D919C911797019617969C938E932D
:100A90001697DA019C91892F869586958927837010
:100AA000DF01AA53BF4F833039F48C91803214F4A4
:100AB0008F5F01C081508C938C91885F803414F4D7
:100AC0008C9346C18F738C93DF01A953BF4F8C91D8
:100AD000880F97702BEF290F233010F0933009F413
:100AE00081608C938C91982F969589278095817041
:100AF0009685990F892B86878E3709F048C0DF01CC
:100B0000AB58BF4F14962D913C9115978D919C91A8
:100B100011972817390761F416962D913C91179774
:100B200012968D919C9113972817390709F4DCC010
:100B300016962D913C91179714968D919C9115972F
:100B400001972817390709F4CFC01696CD91DC918B
:100B500017978EE7888316962D913C9117971296DA
:100B60008D919C9113972817390721F48D919C91B1
:100B7000119705C016968D919C911797019617961F
:100B80009C938E93169781E0818B2A9AB0C0982F00
:100B90009F779F3719F4118A2A98DAC0918999238F
:100BA00009F4D6C0982F9F739E3309F4D1C080FFFB
:100BB00003C080898068808B97859F5F9787808935
:100BC000983008F499C0DF01AB58BF4F92E8980FF6
:100BD000923018F08B3109F044C014962D913C915D
:100BE00015978D919C9111972817390759F41696EE
:100BF0002D913C91179712968D919C9113972817E0
:100C0000390759F116962D913C91179714968D91AD
:100C10009C911597019728173907F9F01696CD91F1
:100C2000DC9117978BE1888316962D913C9117974D
:100C300012968D919C9113972817390721F48D9165
:100C40009C91119705C016968D919C9117970196CE
:100C500017969C938E93169704C0118A2A9880E069
:100C600001C081E014964D915C9115972D913C91B6
:100C700011974217530759F416964D915C911797A7
:100C800012962D913C9113974217530769F11696CE
:100C90004D915C91179714962D913C911597215089
:100CA00031094217530701F190891696CD91DC91D5
:100CB0001797988316964D915C91179712962D91E0
:100CC0003C9113974217530721F42D913C911197B2
:100CD00006C016962D913C9117972F5F3F4F1796A0
:100CE0003C932E93169703C0118A2A9880E0108AAD
:100CF0001786882321F02CC08695808B29C0DF01C0
:100D0000A853BF4F8D919C911197816011969C9330
:100D10008E93EB58FF4F2481358180819181281774
:100D2000390739F426813781828193812817390761
:100D300041F02681378184819581019728173907F1
:100D400039F4868197819583848311961C921E9233
:100D5000DF91CF911F910F91FF90EF9008951F9217
:100D60000F920FB60F9211242F933F934F935F93DF
:100D70006F937F938F939F93AF93BF93EF93FF9363
:100D800080E286BB609178007091790076956795D6
:100D900076956795605880912C0890912D080E9457
:100DA000CD0480911301882349F080912C08909103
:100DB0002D080E94B203807F886001C080E88BB953
:100DC0008091F6049091F704A091F804B091F90491
:100DD0000196A11DB11D8093F6049093F704A09392
:100DE000F804B093F904FF91EF91BF91AF919F91F7
:100DF0008F917F916F915F914F913F912F910F90C4
:100E00000FBE0F901F901895CF92DF92EF92FF9236
:100E10000F931F93CF93DF931F92CDB7DEB77C0163
:100E2000262F82E8860F8701085E1C4F823010F063
:100E30006B3149F4F801608171818BE190E0298385
:100E40000E94BB0A2981D701A25EBC4F3C9111963A
:100E50004C911197822F90E0FC01E327EE0FFF1FCA
:100E6000E851FF4F25913491C42ED12C2C253D25DE
:100E70002D933C93F801608171810F90DF91CF91A8
:100E80001F910F91FF90EF90DF90CF900C94BB0AD1
:100E900024E233E0DC01F9011D923197E9F7FC010E
:100EA000E85EFC4F718360833896518340833297AC
:100EB0002FEF3FEF318320833297318320830895D2
:100EC0003F924F925F926F927F928F929F92AF92DA
:100ED000BF92CF92DF92EF92FF920F931F93CF9327
:100EE000DF932C013C0128EE621A2CEF720A6C0190
:100EF0004DEDC41A4CEFD40AEC01CE5DDC4F8C01F1
:100F0000065E1C4F7C0184EEE81A8CEFF80A33244D
:100F10003394AA24AA94BA2C4201A0EE8A1AACEF08
:100F20009A0AF301808191810E947D0A8F3FFFEF31
:100F30009F0709F458C0F6012081211128C08E377F
:100F40009105D1F4D8018D919C91429768F0F701F9
:100F500080819181883B904F39F4D401ED91FC91CF
:100F6000309711F0C20109953882F701B182A08251
:100F7000D8011D921C92D5CF8F37910511F418829C
:100F8000D0CF8B31910519F4F6013082CACF288178
:100F9000222331F1D8012D913C912831B3E03B0758
:100FA000F0F4A9014F5F5F4FF80151834083F201D4
:100FB000E20FF31F8083D7012D913C91F901E827BF
:100FC000FF27EE0FFF1FE851FF4F85919491232FCC
:100FD000332782279327F7019183808301C01882EA
:100FE000D6011C929ECFDF91CF911F910F91FF9060
:100FF000EF90DF90CF90BF90AF909F908F907F90B9
:101000006F905F904F903F9008958F929F92AF9214
:10101000BF92CF92DF92EF92FF920F931F93CF93E5
:10102000DF938C014B015A016C0182EEC81A8CEFE0
:10103000D80A8FEF9FEFF601918380837801F8EE55
:10104000EF1AFCEFFF0AF701608171818EE790E0F3
:101050000E94BB0AE401A80CB91CCA15DB0529F0E3
:101060006991C8010E940407F8CFF6016081C1812F
:101070006095C8010E9404076C2F6095C8010E940A
:101080000407F701608171818EE790E0DF91CF91D5
:101090001F910F91FF90EF90DF90CF90BF90AF9096
:1010A0009F908F900C94BB0A9093300880932F08E8
:1010B0005093FB044093FA04709332086093310814
:1010C0000895EF92FF920F931F93CF93DF93EC015C
:1010D0006091FA047091FB0480EC90E00E94BB0ADE
:1010E0006091FA047091FB0480E090E00E94BB0ADA
:1010F0008E017E0186EEE81A8CEFF80AF701208156
:101100003181225031096091FA047091FB04C801C9
:101110008C1B9D0B8217930708F5F80181918F01B5
:10112000803C59F48BED90E00E94BB0A6091FA0478
:101130007091FB048CED90E00EC08B3D59F48BED6B
:1011400090E00E94BB0A6091FA047091FB048DED5F
:1011500090E001C090E00E94BB0AD0CF80EC90E00C
:10116000DF91CF911F910F91FF90EF900C94BB0AEC
:101170004F925F926F927F928F929F92AF92BF92A7
:10118000EF92FF920F931F93CF93DF93EC018B01AC
:101190007A01E0913108F09132088189811145C0CE
:1011A0000E946D0A90910001891798F4A701B80177
:1011B000CE01DF91CF911F910F91FF90EF90BF90E3
:1011C000AF909F908F907F906F905F904F900C9416
:1011D00005088FB7F8948090F6049090F704A090DB
:1011E000F804B090F9048FBF209101013091020101
:1011F0004091030150910401AAE0B0E00E94F4097B
:101200002FB7F8944090F6045090F7046090F804DB
:101210007090F9042FBF481859086A087B084616D1
:1012200057066806790664F3B4CFE0913108F0916F
:1012300032088189882309F4ACCF80912F089091DE
:1012400030080E946007E0913108F0913208E853BD
:10125000FF4F80819181892B41F311821082DF91B0
:10126000CF911F910F91FF90EF90BF90AF909F9003
:101270008F907F906F905F904F900895909133087A
:101280009923A1F0803C01F580910D01811111C0DD
:1012900010923308409134085091350864E171E0B0
:1012A00080912F08909130080C94B808803C09F088
:1012B0007BC081E0809333088EEF80930D01109204
:1012C000350810923408089520913408309135087B
:1012D000283193E0390708F067C090910D0121157E
:1012E000310531F49E3F21F48F7080930D010895F4
:1012F00091111FC08B3D21F481E080932E08089549
:1013000090912E08992349F08C3D21F08D3D19F4E0
:101310008BED01C080EC10922E08A9014F5F5F4F4A
:101320005093350840933408F901EC5EFE4F8083FA
:101330000895913079F4282F30E0AAE0B0E00E94BF
:10134000E5096093090170930A0180930B01909362
:101350000C010895943089F42AE0829FC001112481
:10136000AA2797FDA095BA2F8093050190930601B7
:10137000A0930701B09308010895933089F42AE0FF
:10138000829FC0011124AA2797FDA095BA2F8093B0
:10139000010190930201A0930301B0930401089509
:1013A000923011F48093000108950E94950188E025
:1013B00095E00E94600780E00E9404028823B9F350
:1013C0000E940E020E943E09F2CFA29FB001B39F7D
:1013D000C001A39F700D811D1124911DB29F700D3E
:1013E000811D1124911D08950E94E509A59F900D6E
:1013F000B49F900DA49F800D911D11240895A1E22A
:101400001A2EAA1BBB1BFD010DC0AA1FBB1FEE1F7E
:10141000FF1FA217B307E407F50720F0A21BB30BC9
:10142000E40BF50B661F771F881F991F1A9469F745
:1014300060957095809590959B01AC01BD01CF01A1
:1014400008958F929F92AF92BF92CF92DF92EF92C8
:10145000FF92CF93DF93EC01688179818A819B8130
:10146000611571058105910521F464E279ED8BE543
:1014700097E02DE133EF41E050E00E94FB0A490183
:101480005A019B01AC01A7EAB1E40E94F4096B0187
:101490007C01ACEEB4EFA50194010E94F60ADC01D8
:1014A000CB018C0D9D1DAE1DBF1DB7FF03C0019765
:1014B000A109B04888839983AA83BB839F77DF9172
:1014C000CF91FF90EF90DF90CF90BF90AF909F9023
:1014D0008F9008950E94210A08958EE091E00E9465
:1014E000210A0895A0E0B0E080930E0190930F01CF
:1014F000A0931001B09311010895CF93DF93EC01F5
:101500002B8120FF33C026FF0AC02F7B2B838E81C7
:101510009F8101969F838E838A8190E029C022FF5C
:101520000FC0E881F9818081992787FD9095009708
:1015300019F420622B831AC03196F983E8830EC018
:10154000EA85FB85099597FF09C02B81019611F06B
:1015500080E201C080E1822B8B8308C02E813F8115
:101560002F5F3F4F3F832E83992702C08FEF9FEF5E
:10157000DF91CF9108950F931F93CF93DF93FB01DA
:10158000238121FD03C08FEF9FEF28C022FF16C0EB
:1015900046815781248135814217530744F4A08145
:1015A000B1819D012F5F3F4F318320838C93268132
:1015B00037812F5F3F4F3783268310C0EB01092F00
:1015C000182F0084F185E02D0995892BE1F68E8195
:1015D0009F8101969F838E83812F902FDF91CF91E2
:1015E0001F910F910895B7FF0C94F4090E94F4091C
:1015F000821B930B0895052E97FB1EF400940E9406
:10160000120B57FD07D00E94FF0907FC03D04EF4D0
:101610000C94120B50954095309521953F4F4F4FAC
:101620005F4F089590958095709561957F4F8F4F8E
:081630009F4F0895F894FFCFCD
:101638003FC8000000320000005E010000FE01000B
:021648000000A0
:00000001FF
